:020000040000FA
:02000000702866
:08000800332BA3002308122092
:10001000A400FF302402031D0E2808002408D42267
:10002000A30A0628A0000A30A00200308A00200897
:100030001C3E03188A0A82005034613474346934D7
:1000400065346E34743465347A342034FF34453486
:10005000543441344C344F344E344E3441344734AC
:10006000453420344D3441344E34433448344534DF
:100070005334FF3445344D34443420343234303436
:10008000303438342034FF34543465346D347034B3
:1000900020344D344F3454344534553452342034A4
:1000A00031343A34FF34543465346D347034203490
:1000B0004D344F3454344534553452342034323472
:1000C0003A34FF34543465346E34733469346F34E5
:1000D0006E34203461346334633475343A34FF341D
:1000E0000313831600309F008710071007110610B6
:1000F0008610061186110616861681138130990026
:100100001812181598168C160C140313831231301C
:10011000900081309F00FA302223FA30222387108A
:100120000710071106108610061186110614861492
:10013000EF220F302223EF220F302223EF220F3045
:10014000222306108614EF222830C2220C30C2224D
:100150000630C222BD22AD01AF01B001B1010030B5
:10016000B200B300B400B500B600B7009817181677
:100170000B178B17BD228630C2220A30052095301E
:10018000C222153005209F151F169F12B622A90006
:100190009F111F169F12B622AA009F151F129F12B1
:1001A000B622AB002A23BD228130C2223230052084
:1001B000C130C222413005209530C2225030052086
:1001C000E030C222283005201430BB009F151F16D6
:1001D0009F12B622A5002908A5029F111F169F1283
:1001E000B622A7002A08A7029F151F129F12B62247
:1001F000A6002B08A60206083039A8000310A80C98
:10020000A80CA80CA80C2430B2225430B2224330DF
:10021000B2222508B2222608B2222708B2222808D4
:10022000B222AE1C172994219B21A2211D29303016
:10023000B200B300B400B500AF0121213B2155212C
:10024000E6283208303C031D32293308303C031DB8
:1002500032299030C2222030D4222030D4222030C3
:10026000D42208009030C2223208D4223308D4228B
:10027000DF30D42208003408303C031D4C293508F7
:10028000303C031D4C29D030C2222030D4222030F3
:10029000D4222030D4220800D030C2223408D42204
:1002A0003508D422DF30D42208002F08031D652929
:1002B000A330C2222030D4222030D4222030D422B5
:1002C0002030D4222030D42208004C3036020319CA
:1002D0007A294830360203198729A330C22236080A
:1002E000D4222C30D4223708D4225630D4222030C5
:1002F000D4220800A330C2224230D4224130D4227A
:100300005330D4225330D4224530D4220800A330B5
:10031000C2224830D4224130D4225530D422543025
:10032000D4224530D422080030089B223908B2007C
:100330003A08B300080031089B223908B4003A0893
:10034000B50008004D302F02031C132A4E302F0237
:10035000031C182A4F302F02031C1D2A51302F0274
:10036000031C222A52302F02031C272A53302F024B
:10037000031C2C2A54302F02031C312A56302F0222
:10038000031C362A57302F02031C3B2A58302F02F9
:10039000031C402A5A302F02031C452A5B302F02CF
:1003A000031C4A2A5C302F02031C4F2A5D302F02A7
:1003B000031C542A5F302F02031C592A60302F027D
:1003C000031C5E2A61302F02031C632A63302F0254
:1003D000031C682A64302F02031C6D2A65302F022B
:1003E000031C722A66302F02031C772A68302F0202
:1003F000031C7C2A69302F02031C812A6A302F02D9
:10040000031C862A6C302F02031C8B2A6D302F02AE
:10041000031C902A6E302F02031C952A4830B60028
:100420004830B7009A2A4C30B6004C30B7009A2AB0
:100430003630B6003030B7009A2A3630B600313048
:10044000B7009A2A3630B6003230B7009A2A3630D2
:10045000B6003330B7009A2A3630B6003430B700D1
:100460009A2A3630B6003530B7009A2A3630B600B0
:100470003630B7009A2A3630B6003730B7009A2A9D
:100480003630B6003830B7009A2A3630B6003930E8
:10049000B7009A2A3730B6003030B7009A2A373082
:1004A000B6003130B7009A2A3730B6003230B70084
:1004B0009A2A3730B6003330B7009A2A3730B60060
:1004C0003430B7009A2A3730B6003530B7009A2A50
:1004D0003730B6003630B7009A2A3730B60037309A
:1004E000B7009A2A3730B6003830B7009A2A37302A
:1004F000B6003930B7009A2A3830B6003030B7002D
:100500009A2A3830B6003130B7009A2A3830B6000F
:100510003230B7009A2A3830B6003330B7009A2A02
:100520003830B6003430B7009A2A3830B60035304B
:10053000B7009A2A0800B801B901BA01BA006430BC
:100540003A02031CA62ABA00B80A9F2A0A303A02C5
:10055000031CAD2ABA00B90AA62A3030B807B90779
:10056000BA0708000C1EB22A9900080005302223A1
:100570001F151F19B92A1E0808000130C2220130B8
:1005800022230800A100F62207102108A200A100E2
:10059000A20CA20CA20CA20C2208DA22EF22210843
:1005A000A200DA22EF220800A100F6220714210897
:1005B000C62208002218DE2A0610DF2A0614A21816
:1005C000E32A8610E42A86142219E82A0611E92A69
:1005D0000615A219ED2A8611EE2A86150800871441
:1005E00000000000000000008710080003138316BD
:1005F00006148614061586150313831207100715B3
:10060000871400000608A20087100000871400006D
:10061000060887100000A219F62A03138316061095
:1006200086100611861103138312071108000A3081
:10063000FB00FB0B1C2B212BB630FC00FC0B1E2BF4
:10064000192B0800FD00FD0AFD0B272B292B172372
:10065000242B0800FA302223FA302223FA302223F6
:10066000FA3022230800FF000308FE000313831260
:100670000C1C472B0C102E1C3F2B2E10432BBB0B9E
:10068000752BAE10752BAE141430BB00752B2E14C9
:100690001A08AC002D18522B24302C02031D752B88
:1006A0002D14752BAD185A2B54302C02031D742BAE
:1006B000AD14752B2D19622B53302C02031D732B97
:1006C0002D15752BAD19682B2C08AF00AD15752BAA
:1006D0002D1A6E2B2C08B0002D16752B2C08B1008E
:1006E0002D12AD112D11AD102D107E088300FF0EBF
:0406F0007F0E090070
:084000000100090004000900A1
:02400E00323F3F
:00000001FF
